:020000040000FA
:020000000528D1
:08000800402900308B00850146
:100010008601831611308500023086008312831614
:100020006730990098161815181283129817181629
:100030008C1283168C1683120B178B1707309F00B8
:10004000FF30A500B101B001B101AA01AB01AC01C3
:10005000AD01AE01AF30A600AF30A700AF30A800B1
:10006000AF30A900061286120613861386150610F5
:100070008513722186113D203B28851426086221B4
:1000800085100515270862210511851528086221AC
:10009000851105172908622105136D21080006083E
:1000A0000F398600301C5628061657280612B01C39
:1000B0005B2886165C288612301D6028061761288A
:1000C0000613B01D65288617662886130800051CD0
:1000D0006B2831106C283114051E7028B11071285E
:1000E000B114851E7528311176283115080053305A
:1000F000990059213108303E9900592108002F1CE0
:10010000822888282508453A031D08002F14080076
:100110002508533A0319B92825084D3A0319F1283F
:100120002508423A03192B2925084C3A0319362988
:100130002508523A031923292508463A0319332979
:10014000AF1CA9282F1DAD28AF1DB1282F1EB52823
:1001500008002508AA00AF1408002508AB002F15D9
:1001600008002508AC00AF1508002508AD002F16C3
:1001700008003030AA023030AB023030AC023030F0
:10018000AD022B08AE006330A4002E08AB07A40B11
:10019000C5282C08AE000930A4002E08AC07A40B1B
:1001A000CD282B082C072D07AE002A08013A031D85
:1001B000DC282E08A600F0282A08023A031DE328AE
:1001C0002E08A700F0282A08033A031DEA282E0863
:1001D000A800F0282A08043A031DF0282E08A900D8
:1001E0003E293030AA023030AB023030AC02303021
:1001F000AD020310AA0DAA0DAA0D0310AB0DAB0D95
:100200000310AC0DB1013008B100B0012A08B004F0
:100210002B08B0042C08B0042D08B0043008093AAB
:10022000031D13291F293008063A031D18291F2909
:100230003008003A031D1D291F293108B00030087D
:10024000B1004F203E293030AD022D1C29298517E1
:10025000322985133E293030AD022D1C31298615F7
:10026000322986113E29672077203E293030AD02A1
:100270002D1C3C2906143D2906100000AF01080082
:10028000B3000308B5000A08B4008C1E52290630DA
:100290001805031D4F291A08A5007F20532918129D
:1002A00018165329522934088A0035088300330868
:1002B00009008316981C5A29831208002508990002
:1002C00059210800A000000000000000000000000C
:1002D00000000000A00B632908001830A0000030C7
:1002E000A3007C290830A2000130A300FF30A00049
:1002F0002318A20B7C290800AA30A100A10B7E299B
:0A030000A00B7C29231876290800C1
:02400E00183F59
:00000001FF
